:100000009F01831691010730831299003F308316B8
:1000100085003F30870002308312A3006F148316DF
:10002000871607168312960116179616161597014E
:10003000971717171716971191019115A701A4018A
:100040000730930092016F11EF108C1E25281718AE
:10005000EF141408A500EF1C392823082502031DFE
:10006000362897115A30A6006F1537289715A70123
:10007000EB2800308A0027083E3E82004228D8281C
:10008000DF28E62800308A00250EB600B60C360CB4
:1000900003394B3E82004F28D728D728A5280030A7
:1000A0008A00250CB600B60C360C0739583E820083
:1000B0006028A4288A288B288C288C2897289728A1
:1000C00000308A0007302505663E82006E287228BF
:1000D00078287C2881288528892889284121A6001C
:1000E0006F1589284121A6006F150130A7008928C6
:1000F0007021A6006F1589280230A700A6016F1590
:1001000089281A21A6006F1589280330A700A601A7
:100110006F15A428A428A4284121A6006F15F0304B
:100120002605B6000F30250536045821A4284121A4
:10013000A6006F150F302605B6000F302505B70055
:10014000B70EF03936045821D72800308A00250C24
:10015000B600B60C360C0739AE3E8200D728D72839
:10016000D728D728D728D728D728B62800308A00FC
:1001700007302505BC3E8200D728D728D728D728A6
:10018000C428C528D028D428D7286F15A6011A302E
:1001900024020318CF282408F120A600A40AD72897
:1001A000A401A6016F15D728A6016F159715EB2896
:1001B000250858214121A6006F15A701EB28250825
:1001C0008B212508A6006F15A701EB2825082F21F4
:1001D000A6016F15A7016F1DF0282608D721B821A9
:1001E0002328840001308A000408003E82000000B9
:1001F00000000000000000000000000000000000FF
:10020000103400340334013403340C344D34693475
:10021000643469346D346F3474346F34723432340E
:100220002D34413407344734723461346D347334BF
:100230006F346E34A8018316111828149118A8146D
:10024000111928159119A815111A2816911AA8160E
:10025000111B2817911BA817831228080800A90052
:1002600029181114A918911429191115A9199115F2
:10027000291A1116A91A9116291B1117A91B9117D2
:1002800000340508AA000708AB00AC012A182C149A
:100290002A1AAC14AA182C152A19AC152B182C16CE
:1002A000AB18AC162B192C17AB19AC172C0808007F
:1002B000AF00AD01AE012F182D14AF182D162F1958
:1002C000AD14AF192D152F1A2E14AF1AAE142F1B03
:1002D0002E15AF1BAE152D0885002E0887000034A3
:1002E000B201831605088312B00083160708831233
:1002F000B10030183214301AB214B0183215301957
:10030000B21531183216B118B21631193217B119A7
:10031000B21732080800B500C030B300C030B400D6
:1003200035183314B51833163519B314B5193315F8
:10033000351A3414B51AB414351B3415B51BB4155D
:10034000B4163416330883168500831234088316D6
:10035000870083120034FF30B800FF30B9008C1ED4
:10036000B32914080800B90BAF29B80BAD29FC3428
:100370008C1EB82914080800A000200E0F39C421D3
:100380000F302005C4210034A1000A3021020318D7
:100390003730031C3030A1072108D721003420302A
:1003A000D72100340D30D7210A30D7210034A200E4
:0A03B0008C1CD829220895000034A7
:02400E00D230AE
:00000001FF
